:1000000096C0AFC0AEC0ADC0ACC02CC2AAC0A9C023
:10001000A8C0A7C0A6C0A5C0A4C0A3C0A2C0A1C0BC
:10002000A0C09FC09EC075C576C577C578C579C587
:1000300078C577C576C578C587C590C5A1C591C572
:1000400093C597C59BC5B0C5B2C5CCC5CEC5D0C5F7
:10005000CFC5CEC5CDC5D0C52DC6D8C52BC6D9C533
:10006000DAC5E7C5EBC526C625C624C623C622C603
:1000700021C620C61FC61EC61DC61CC61BC61AC664
:1000800019C618C617C614C612011001FF000008D1
:10009000C016B30620460102000134035500530088
:1000A000420032004C005000540020006C006F00F1
:1000B00077002D007300700065006500640020006B
:1000C0006100640061007000740065007200240328
:1000D00068006100660074006D0061006E006E00D3
:1000E000230073006F0066007400770061007200E7
:1000F0006500040309040902370001010080320988
:1001000004000002FF0000000705010208000007CC
:100110000581020800000904000102FF0000000739
:1001200005010308000A0705810308000A001124DD
:100130001FBECFE5D4E0DEBFCDBF10E0A0E6B0E04B
:10014000E6E9F1E102C005900D92A436B107D9F7B6
:1001500010E0A4E6B0E001C01D92AD3EB107E1F7AA
:1001600032C74ECFCF93C62FDC018091C0008E31B5
:10017000E9F08091C00084FF07C08091C10098E839
:1001800089278093C10003C08AE58093C000E2EC18
:10019000F0E09C2F8D91819391501916DCF36C2F18
:1001A00082EC90E05BD1CC5FC093C000CF9108950A
:1001B0000F931F93CF93DF93C091D200C350C7FD1D
:1001C000D4C08091CE0002EE10E0081B110980918E
:1001D000CD008D3211F48AEF5FD48091CD00803153
:1001E00020F46C2FC801D9D6BAC08D3209F0A6C050
:1001F000C83009F0B4C083EC8093B4005AE5509342
:10020000600010926400E8019881892F807621F0C7
:10021000C8015ED5982F7DC0382FEDEBF0E0E801E6
:100220002A814C818093BD008981882381F49F714C
:10023000923051F4413841F4932F8091C0008E31B7
:1002400009F491E09093BD00118232E05DC08130ED
:1002500011F0833089F4222309F056C0413809F0A7
:1002600053C0813011F4852F01C08EE18093C0000E
:100270008BE48093C10048C0853019F42093D300EB
:1002800043C0863049F5F8018381813021F432E1A1
:1002900088E890E019C0823021F437E386EF90E0DF
:1002A00013C08330A9F4222321F434E082EF90E0DC
:1002B0000BC0213021F434E28EEC90E005C02230F6
:1002C00039F434E38AE990E09093D1008093D00030
:1002D00080E4809364001CC0883019F4E5EDF0E000
:1002E00009C0893029F42093D5005093C0000CC078
:1002F0008A3011F431E008C08B3031F48BE4809304
:10030000C1008AE58093C000F093D100E093D00053
:10031000932F9F3F41F4E801888187FD9E8180E80B
:100320008093640008C0F8018781882321F48681C6
:10033000891708F4982F9093610011C08091640090
:1003400087FF0DC06C2FC801CDD58F3F21F48EE102
:100350008093600004C0882311F0109261008091A6
:10036000D200181614F41092D2008091600084FF1D
:1003700044C0809161008F3F09F43FC0682F8930ED
:1003800008F068E0861B809361008091B40098E8D3
:1003900089278093B400A5EBB0E06623E9F0809153
:1003A000640087FF04C0CD0150D5682F15C0962F7B
:1003B000E091D000F091D10086FF06C084918D932A
:1003C00031969150D9F704C081918D939150E1F706
:1003D000F093D100E093D0007727C62F693038F42E
:1003E00085EB90E03BD0CC5FCC3028F401C0CEE16F
:1003F0008FEF80936100C093600094E186B38370B7
:1004000049F49150D9F79093D3009093CC008AE5AA
:100410008093C000DF91CF911F910F91089589B70C
:10042000806289BF8BE48093C1008AE58093C0001D
:100430000895A82FB92F80E090E041E050EA609540
:100440006F5F58F42D9138EF82279795879510F0BC
:10045000842795273F5FC8F3F3CF0895EADF8D9394
:100460009D930895CF93CFB7CF93C395B09BE9F7F2
:10047000B09B20C0B09B1EC0B09B1CC0B09B1AC0DC
:10048000B09B18C0C091CF00C395C093CF00DF933D
:10049000C2B7D091EC00C093EC00CD1BC85CD1B7C3
:1004A000C23012F0D15003C0CF3F0AF4D395D1BF70
:1004B000DF9148C1DF93C091CE00DD27CA52DF4FE4
:1004C000B09B02C0DF91D4CF2F930F931F9320E8EE
:1004D000B09921604F933F930F92B09922601FEF24
:1004E0003BE0022F220F00C0B0990C60202708705B
:1004F00046B311F4000036C0B4C040FFC89546B3FF
:10050000206800000227B09B0AC0287F11F046B384
:1005100088C046B31E7FB09BB19901C06AC040FD40
:10052000C89546B321604370B09908C0B9F3217FE4
:1005300046B309F087C01D7F00C000C040FFC895CA
:1005400046B322600000B09B08C0237E11F046B382
:1005500087C046B31B7F00C000C040FDC89546B3AE
:1005600024600993B09908C0277C11F046B387C076
:1005700046B3177F00C000C040FFC89546B328604F
:10058000012FB09B08C02F7811F046B387C046B347
:100590000F7E00C000C040FDC89546B320611FEF2C
:1005A000B09908C02F7111F046B387C046B30F7DD4
:1005B00000C000C040FFC89546B32062315038F0FB
:1005C000B09B08C02F73223046B314F085C08EC094
:1005D0000F7BC89540FDC89546B320640000B099D4
:1005E0008CCF2F77243046B30CF00AC00F77000071
:1005F00084CF09937FC040FDC89546B320680000B2
:100600000227B0990AC0287F11F046B38CCF46B3B9
:100610001E7FB09BB19901C0ECCF40FFC89546B397
:1006200021604370B09B09C0217F19F046B30000E0
:100630008ACF46B31D7F00C000C040FDC89546B3B9
:10064000C1F22260B09908C0237E11F046B389CF71
:1006500046B31B7F00C000C040FFC89546B324606E
:100660000993B09B08C0277C11F046B389CF46B3ED
:10067000177F00C000C040FDC89546B32860012F19
:10068000B09908C02F7811F046B389CF46B30F7EDA
:1006900000C000C040FFC89546B320611FEFB09B6B
:1006A00008C02F7111F046B389CF46B30F7D00C04B
:1006B00000C040FDC89546B320623150B8F0B099F3
:1006C00007C02F73223046B30CF089CF0F7BC8953B
:1006D00040FFC89546B32064B09B8DCF2F77243060
:1006E00046B30CF00FCF0F77000085CF10E218BF94
:1006F00000271CC03B503195C31BD04010E218BFEF
:100700000881033C19F10B3409F12091CC001981C7
:10071000110F1213EDCF4A81441F093671F10D32CA
:1007200011F0013E29F74F7009F0042F0093D40017
:100730000F903F914F911F910F912F91DF91C8B76B
:10074000C5FD93CECF91CFBFCF9118952091D40006
:10075000222371F31091D200112379F534307AF10C
:100760000093BF003093D2002093CD001091CE00B3
:100770003BE0311B3093CE0022C00091D20001300B
:10078000E4F40AE54F7049F43091600034FD18C07C
:1007900000936000C4EBD0E017C03091C00034FD7E
:1007A0000FC00093C000C1ECD0E00EC0279598F4B4
:1007B000415099F4220F0000F9CF3AE501C032ED23
:1007C000032EC0E0D0E032E017B31360C09A17BB2D
:1007D00008B320E413E0012746E008BB279520F486
:1007E000415021F4220FF9CF012746E0000000001C
:1007F0003B5A08BBD8F2279528F4415029F4220F20
:100800000000F9CF012746E0279508BB20F44150AE
:1008100021F4220FF9CF012746E02991000033236C
:1008200008BB21F60C7F1091D300110FC250D040AD
:1008300008BB11F01093CC0010E218BF016017B391
:100840001C7F402F4C7FC895C89508BB17BB48BB81
:100850006FCF3091680031FD16C020916D00E22FFE
:10086000FF27EE0FFF1FE151FF4F918380832F5F22
:100870002F703E7F80916C00281709F4326020931E
:100880006D0030936800089520916C0030916800ED
:1008900030FF0CC021502F70E22FFF27EE0FFF1FFB
:1008A000E151FF4F0190F081E02D15C0E22FFF27AD
:1008B000EE0FFF1FE151FF4F2F5F0190F081E02D00
:1008C0002F703D7F80916D00821709F43160209375
:1008D0006C0030936800CF0108958091670085FF18
:1008E00004C011BA8FEF82BB08958091660082BB6D
:1008F00080916B0080FF03C082B3809501C08FEFB1
:1009000081BB0895EADF81E084BB8EE385BB8091E3
:1009100067009BE08927880F880F806C88BB8CE379
:1009200087BB0895982F31B328B39D990CC0822FAF
:10093000892388BB92FD02C08FEF81BB88E19D991E
:1009400007C08150E1F780916A00816080936A005E
:1009500080B392FF31BB28BB99270895982F8091CF
:1009600069008C7421F0892F992773DF0895909383
:1009700066008091670085FD07C092BB80916B0087
:1009800080FF02C0909591BB0895CF93909169002C
:100990009570C82FC06C9111CF7D909167009C27F6
:1009A000C093670080916B0086FD04C095FD95DFC4
:1009B0008BE0C827CC0FCC0F8C2F806C88BB80912C
:1009C0006B0082FF03C0C095CC73C7BBCF91089565
:1009D000282F887F85608093680022952695277050
:1009E00081E090E002C0880F991F2A95E2F7282F36
:1009F00080936900332724FF02C08EEF01C08FEF80
:100A000080936A0025703070232B41F0809167003D
:100A100085FF04C08F7D809367005FDF10926D00BB
:100A200010926C000895809169008C7411F02CDF95
:100A300001C080B39927089593B3990F990F9760D8
:100A400080916B0086FD02C080E8982780916A0043
:100A50009823892F99270895809169008C7411F04B
:100A600088B301C086B3982F969596959F70809114
:100A70006B0086FD02C08BE0982780916700807F25
:100A8000982B892F99270895882329F09FE09A951C
:100A9000F1F78150E1F70895982F80916E00882337
:100AA00019F490937000A89A90936F0090936E0041
:100AB0000895CF92DF92EF92FF920F931F93CF93FF
:100AC0008C01C62F6A017A01662339F480E090E038
:100AD000F7C0806180936500F0C084E6DDDF80911F
:100AE0006500882329F08F7E10926500CF5F03C0D8
:100AF000F80181918F0184FF47C02FEF9927AA2722
:100B0000BB27FC017097E031F105D0F5ED5EFF4F9A
:100B1000099489DF27C090DF25C09EDF23C08FEDB9
:100B200001C087EFFFDE1EC0809169008C7C19F444
:100B30002FEF30E025C087FF03C020E130E020C068
:100B4000A3DE282F33271CC08091690087FF03C0D4
:100B500080E090E007C08FEF90E004C02091680033
:100B60000FC081B3282F0CC024B3220F220F287F7F
:100B700007C027B3269526952F7002C020916B00E1
:100B8000F70121937F0196C0C15009F4A2CFF8016B
:100B900021918F019927AA27BB27FC01819708F093
:100BA00089C0ED5DFF4F0994822FD8DE83C080910C
:100BB000690084FF07C020FD05C080916A008E7F18
:100BC00080936A00922F9695969580916B0086FD92
:100BD00005C080E2982784B38095982B9E7385B3D7
:100BE000817024C0822FD1DE65C022BB8BED02C094
:100BF00022BB83EF97DE5EC0809169008C7409F49C
:100C000059C0822F9927916024DE54C0822FE0DEE4
:100C100051C021BB4FC0922F96959695916C94BB75
:100C200080916B0086FD46C0909585B3892B85BB6E
:100C300041C0220F220F2C7327BB3CC0622F65746A
:100C400080916B00862760936B00882399F1482F71
:100C5000552740FF12C0262F3327C901807490709A
:100C6000892B59F48091670085FD07C020FF03C0E0
:100C700082B3809501C08FEF81BB42FF0FC0262F4A
:100C80003327C90180749070892B41F422FF04C07E
:100C900088B380958C7301C08CE387BB46FF0AC084
:100CA000862F992780749070892B21F42BDE02C047
:100CB000822FEADEC15009F012CF8E2D8C199927B0
:100CC000CF911F910F91FF90EF90DF90CF900895FB
:100CD000FC0181818093B100828193819093B30064
:100CE0008093B200868197819093110180931001C7
:100CF0008DEE90E09093D1008093D000208122303F
:100D000069F48181833051F48281882339F48481AC
:100D1000813021F483EC8093620094C09181992307
:100D200049F482818093ED0083818093EE0082E01C
:100D300090E00895913091F48281882311F473DE5C
:100D400003C0813031F478DE8093ED0081E090E0E3
:100D50000895823009F076C07FDEF6CF923061F4DC
:100D60008281882319F48481F9DD6CC0823009F016
:100D700069C084810ADE66C0203C09F045C0692F45
:100D80006059653030F580910F0199278F589F4F3A
:100D9000AC01CF0102968DDE20910F01280F209328
:100DA0000F0181EA8093B10081E790E09093B30056
:100DB0008093B20033278091100190911101281780
:100DC000390720F4309311012093100110920F0184
:100DD00039C0892F815A8330A8F5933A81F58091E3
:100DE000B2009091B300069751F520911001309117
:100DF00011012230310519F588ED9AE39093EE0048
:100E00008093ED00C90108952034E1F4692F605901
:100E1000653090F480910F0199278F589F4FAC0156
:100E2000CF01029646DE90910F01980F90930F012B
:100E300080E98093B10006C0915A923018F48FEF88
:100E400090E0089580E090E008951F93CF93DF93A2
:100E5000FC01162FC091B200D091B300262F33278A
:100E600080911001909111018217930710F4109155
:100E700010018091B100813A39F4812F9927AC019A
:100E8000BE01CF016BD117C0823A49F4812F992757
:100E9000DE0101971CF06BD10192FBCF0CC0833AAD
:100EA00039F4812F9927AC01BE01CF014ED103C087
:100EB0002FEF30E012C0212F3327C20FD31FD09362
:100EC000B300C093B2008091100190911101821B78
:100ED000930B9093110180931001C901DF91CF9181
:100EE0001F910895FF920F931F93CF93DF93FC01FF
:100EF000F62EC091B200D091B300262F33278091F7
:100F00001001909111018217930710F4F0901001D5
:100F10008091B100813A49F40F2D1127A801BF013A
:100F2000CE011CD1C00FD11F21C0823A59F490E0EC
:100F30009F15E0F48191DE01082E21D1A89521961C
:100F40009F5FF6CF803979F480910F0199278F58F0
:100F50009F4FAC016F2DCF01ACDD90910F01980F29
:100F600090930F0103C02FEF30E010C0D093B30077
:100F7000C093B2002F2D3327809110019091110161
:100F8000821B930B9093110180931001C901DF9193
:100F9000CF911F910F91FF900895FC018091620005
:100FA0002091BF00281771F488E828272093620059
:100FB00041E750E0CF017DDD682F882319F081E7FC
:100FC00090E0D0D80895CFE5D4E0DEBFCDBF10E0EB
:100FD00094B714BF479A83E083BF85B7806885BF05
:100FE00093FF0BC086B3992783709070892B29F0EB
:100FF00085B78F78806285BF889511DA7894ABEFDA
:10100000BFEFB5D0802D992780936B008F3F11F4EF
:1010100010926B00AAEFBFEFAAD0802D99278823EA
:1010200019F08F3F09F081BF109266008CEC80931D
:10103000670068DC80E2CCDCC09169008C2F9927C6
:1010400082FF0CC08091680080FD3DC09D993BC02F
:101050001BDC82BBC29881E017DD2CC083FF2CC053
:101060008091670085FF12C08091680081FD2BC0D0
:10107000C39903C09C9927C0C39A9C9B24C080B38A
:1010800099279D999160E5DBC3981DC0C29B10C054
:101090008091680080FD17C09D9915C0F5DB82BB6B
:1010A00028B324738070892B09F0286028BBC2986C
:1010B0009D9B09C0C29A07C086B399278370907020
:1010C000892B09F08895C091CF001C1731F486B3A5
:1010D000992783709070892B09F4A89569D81C17FB
:1010E00009F4AACF1C2F20916E00222389F0809151
:1010F0007000815031F485B391E0892785BB8091E0
:101100006F00215009F4A89820936E00809370001E
:10111000E19992CFABEFBFEF2AD0802D90916B0079
:10112000891729F0ABEFBFEF092E29D085CFAAEFA1
:10113000BFEF1DD0902D81B7981709F47DCFAAEF8E
:10114000BFEF81B7082E1BD077CFFB01DC0102C0B7
:1011500005900D9241505040D8F70895FB01DC01F5
:1011600002C001900D9241505040D8F70895E19986
:10117000FECFBFBBAEBBE09A11960DB20895E199C8
:10118000FECFBFBBAEBB0DBA11960FB6F894E29A74
:10119000E19A0FBE08955AFFC300FFFFFFFFFFFF54
:0C21F000FFFFFFFFFFFFFFFFFFFFF200FB
:00000001FF
